:100000000C9470010C94B7010C94B7010C94B701D7
:100010000C94B7010C94B7010C94B7010C94B70180
:100020000C94B7010C94B7010C94F3200C94C721E5
:100030000C94AB160C94B7010C94B7010C94B70157
:100040000C94B7010C94B7010C94B7010C94B70150
:100050000C94B7010C9402170C94B7010C94B701DF
:100060000C94B7010C94B7010C94B7010C94B70130
:100070000C94B7010C94B7010C94B7010C94B70120
:100080000C94B7010C94B7010C94B7010C94B70110
:100090000C94B7010C94B7010C94B7010C94B70100
:1000A0000C94B7010C94B7010C94B701280001001F
:1000B0000100010000000000000000002A2B2800C1
:1000C0000000000000000000000000000000002907
:1000D000000000002C1E3420212224342627252E47
:1000E000362D3738271E1F2021222324252633337F
:1000F000362E37381F0405060708090A0B0C0D0EAB
:100100000F101112131415161718191A1B1C1D2F76
:100110003130232D350405060708090A0B0C0D0E96
:100120000F101112131415161718191A1B1C1D2F56
:100130003130354C000000000000000000000000DD
:1001400000000000000000007E0F00D4FFFFFFC78A
:10015000000000780403300000000E036900730003
:100160006F00700061006400000020036B006500F8
:10017000790062006F006100720064005F006D0032
:100180006100670070006900650000000403090455
:1001900009025B00030100A0FA0904000001030149
:1001A0000100092111010001224000070581030817
:1001B000000A0904010002030000000921110100E6
:1001C0000122220007058203200001070503032006
:1001D00000010904020001030000000921110100CF
:1001E000012281000705840320000A12011001008A
:1001F00000000803A112000100010203010660FFD4
:100200000961A1010962150026FF0095207508818A
:10021000020963150026FF00952075089102C005AC
:10022000010902A10185020901A10005091901299D
:10023000051500250195057501810295017503815C
:10024000010501093009311581257F950275088165
:100250000609381581257F950175088106050C0A68
:1002600038021581257F950175088106C0C00501FA
:100270000980A101850319012AB700150126B700DD
:10028000950175108100C0050C0901A101850419B3
:10029000012AA002150126A002950175108100C057
:1002A00005010906A101050719E029E71500250147
:1002B00095087501810295017508810105071900EE
:1002C00029FF150026FF009506750881000508190D
:1002D000012905950575019102950175039101C0EC
:1002E00011241FBECFEFDAE0DEBFCDBF04B603FEA0
:1002F00027C08091240290912502A0912602B091FE
:1003000027028730904BA740B04BD1F410922402C3
:1003100010922502109226021092270214BE84B772
:10032000877F84BF0FB6F894A8958091600088619C
:1003300080936000109260000FBEE0E0F8E3099542
:1003400011E0A0E0B1E0EAE5F8E402C005900D920A
:10035000A039B107D9F722E0A0E9B1E001C01D92B0
:10036000A432B207E1F70E94A91D0C94F0230C946B
:10037000000081E0089581E008950C94BB01089588
:100380000C94BF011F93CF93DF9300D000D00F9246
:10039000CDB7DEB749835A836B8330919F01898142
:1003A0009A8131111DC06623B9F02223A9F00E9461
:1003B0001B14182F682F89819A810E94CC136981A0
:1003C0007A81812F0F900F900F900F900F90DF91F7
:1003D000CF911F910C94E4070E94F613182FEFCFD2
:1003E0000E941B1469817A81EDCFFC01262F408188
:1003F00051816281738184810C94C201CF93DF9318
:10040000EC0160E00E94F501BE01DF91CF910C94F8
:10041000C001FF920F931F93CF93DF93E82FF0E07B
:10042000EC54FF4FF490C82FC695C695C695D0E002
:10043000FE01EC5BFE4F0491877010E0082E02C0B5
:10044000159507950A94E2F701701127CC5CDE4FF1
:10045000FE01C491D0E002C0D595C7958A95E2F718
:10046000C170DD270115110519F081EE0E94BA0B4C
:10047000209719F086EE0E94BA0B8F2D0E94A70CD0
:10048000CD2B19F086EE0E94510C012B41F081EE2C
:10049000DF91CF911F910F91FF900C94510CDF9140
:1004A000CF911F910F91FF900895EF92FF920F93BC
:1004B0001F93CF93DF93EC01162F0AE088818823E6
:1004C00009F454C0813009F04EC08981813099F41B
:1004D0007E0122E0E20EF11C8A810E94A70CE70156
:1004E0002196812F815050F3EFE9FFE03197F1F72A
:1004F00000C00000F7CF823041F47E0182E0E80EB8
:10050000F11C8A810E94BA0BEACF833041F47E014C
:10051000E2E0EE0EF11C8A810E94510CE0CF8430A3
:1005200011F02196DDCF2A81229690E080E0AE0185
:100530004F5F5F4F2053330B2A30310548F001974E
:1005400078F2EFE9FFE03197F1F700C00000F7CF54
:10055000089FB001099F700D1124C901860F971FD4
:100560002981EA01E4CF0E940902BACFDF91CF913D
:100570001F910F91FF90EF90089560E00C94550249
:100580008F929F92AF92BF92CF92DF92EF92FF92A3
:100590000F931F936B017C0181E090E0A0E0B0E03D
:1005A0004C015D0104C0880C991CAA1CBB1C4A9517
:1005B000D2F7B501A4014C015D0104C0880C991C5F
:1005C000AA1CBB1C2A95D2F7482959296A297B29DC
:1005D00004C0880F991FAA1FBB1F0A95D2F78A0172
:1005E0009B010C211D212E213F21041715072607F1
:1005F000370789F48C299D29AE29BF29BC01CD017B
:100600001F910F91FF90EF90DF90CF90BF90AF9030
:100610009F908F90089580959095A095B0958C218E
:100620009D21AE21BF21EACF0F93382F262F609155
:10063000DD017091DE018091DF019091E001042FD6
:10064000432F0E94C0020F910C940A130E94391785
:100650000E946515811102C00E9402160C948F053C
:100660000C94920508950C94320381E008950C9443
:100670003503CF93C82F0E9433038C2FCF910C9456
:10068000370308950E94360F0E9441032FEF84E341
:100690009CE0215080409040E1F700C000000C94A5
:1006A00026170F931F93CF93DF93EC0161E00E9415
:1006B000F5018C01BE010E945506882359F1BE0147
:1006C000C8010E94BD01882329F1BE01C8010E9412
:1006D00018098823F9F0BE01C8010E94590988232E
:1006E000C9F0BE01C8010E947C0A882399F08A8162
:1006F000882339F001158CE5180751F00E3D1C4593
:1007000079F0CE01DF91CF911F910F910C94B90137
:100710000E94420380E0DF91CF911F910F910895D5
:100720000E940216F7CF90E080E008950895FC0142
:10073000EE0FFF1FEC5AFE4F859194910895CF93D1
:10074000DF930E94E4070E94B404EC01811520E5C8
:10075000920708F042C0811530E4930708F0BDC04D
:10076000883E910528F5803E910508F09DC0883AA5
:10077000910588F4853A910508F08FC08130910584
:1007800009F492C0009709F48FC0049708F08CC058
:10079000D0E0C0E089C08F3B910508F489C0805C3F
:1007A0009109C03CD105A0F30E949703EC017CC0E5
:1007B0008115904250F4C11581E0D80708F074C04B
:1007C000C03FD10528F3D0656FC0C11590E3D907AC
:1007D00008F079C0CE019F70E7CF811525E592071B
:1007E00058F5811534E5930708F0A6C0811542E558
:1007F000940750F4C11581E5D80708F471C0DC2FC7
:10080000CC27C16FD06A50C0982F969596959E01BF
:1008100023703327C115D34508F07FC0C1E0D0E075
:1008200002C0CC0FDD1F2A95E2F720E2929FC001A3
:100830001124C82BD92B6FC0C11589E5D807A8F49E
:10084000C11598E5D90708F07CC0C11526E5D20787
:1008500008F09ECF8C2F0E944B05C82FD0E0DC2FD4
:10086000CC27CC27DF71D0621FC0C1153AE5D30772
:1008700008F46CC0CE0190568115904208F088CFE4
:100880008D2F8F710E944B0590E0982F8827882725
:100890009F719C012C2BE901E6CFC55AD0E0CD5BBE
:1008A000DE4FC881D0E0D064CE01DF91CF910895B2
:1008B000C85AD0E0CC0FDD1FCB5EDE4F0990D88147
:1008C000C02DD464F1CFCE019927D3FF03C0EC0132
:1008D000D86CEACFEC01D06CE7CFDF70D06AE4CF00
:1008E000CE01E4E096958795EA95E1F783702C2F89
:1008F00026952695237090E2299F90011124382B8C
:100900008C2F8370C1E0D0E002C0CC0FDD1F8A9530
:10091000E2F7C22BD32BDC68C7CFC1E0D0E002C026
:10092000CC0FDD1F2A95E2F730E2939FC00111241E
:10093000C82BD92BDA68B8CFD82FCC27C46FD06A90
:10094000B3CFDC2FCC27C06FD06AAECF8C2F8F7087
:100950000E944B0534E0D695C7953A95E1F7CF70E4
:100960009C2FEC01D069A0CF82389105B1F1B0F491
:100970008133910509F475C048F48932910509F471
:1009800069C08A32910509F473C0089585339105D1
:1009900009F459C08933910501F10895833E910509
:1009A000A9F138F4803E9105F9F0823E910549F1B4
:1009B0000895863E9105A9F1873E9105C9F1843ECF
:1009C000910519F52091160221FF1FC08091150293
:1009D00084FD14C087EE90E00895209115022370E5
:1009E000A1F080EE90E008952091150220FD47C00F
:1009F0003091160230FF09C024FF44C090E080E02F
:100A000004C02091150222FDF7CF08952091150210
:100A100022FD3BC03091160230FDE3CF24FFF5CF1D
:100A2000EDCF2091150223FFF0CF24FDE7CFD2CFE9
:100A30002091150223FD2CC03091160231FFEECF1C
:100A400084EE90E008952091150225FFDECF89E223
:100A500090E008952091150225FFD7CF85E390E01F
:100A600008952091150226FFD0CF8AE290E00895E4
:100A70002091150226FFC9CF81E390E0089589E314
:100A800090E0089583EE90E0089582EE90E008955E
:100A900086EE90E008959091150292FF06C0282FEF
:100AA00028712830F9F4877F846093FF06C0282FCF
:100AB00028712831F1F4877E84612091160220FF8D
:100AC00006C0382F38713830D9F4877F816021FF14
:100AD00006C0282F28712831D1F4877E816194FDCA
:100AE000877E0895282F24712430F9F68B7F886043
:100AF000DCCF282F2471243101F78B7E8861DDCF74
:100B0000382F3171313019F78E7F8860E0CF282F70
:100B10002171213121F78E7E8861E1CF08950C94F7
:100B20008E0508950C949105E82FF0E0E05FFD4FED
:100B300080810895089584988C9A10920F021092E3
:100B4000100281E00E94C7050C942603CF938FB159
:100B500090E024E0959587952A95E1F7809590950A
:100B60008170992720910F02C0E0281719F0809317
:100B70000F02C1E02C2F41E060E172E08FE092E0D3
:100B80000E94C8050E9430038C2FCF9108950895CC
:100B9000FF920F931F93CF93DF93F82E092F162FF9
:100BA000D72FC42F222349F081E0809392010E9425
:100BB000DB1690939101809390018091920188239C
:100BC000A1F080919001909191010E94F3160697F7
:100BD00060F0EF2DF02FA12FBD2FCE0FDF2FD11DF5
:100BE000EC17FD0741F410929201DF91CF911F9114
:100BF0000F91FF90089581918D93F2CF82E290E062
:100C00000E94AE23803289F483E290E00E94AE23FA
:100C1000823159F484E290E00E94AE2391E089325F
:100C200009F090E0892F8170089580E0FCCFCF9388
:100C3000C82F6FEF811160E282E290E00E94BC2336
:100C40006FEFC11162E183E290E00E94BC236FEF7D
:100C5000C11169E284E290E0CF910C94BC2380E062
:100C60000E9417060C945F15089585E290E00E949B
:100C7000AE23682F70E090E080E0089585E290E078
:100C80000C94BC230E9434060E94FE0581110CC006
:100C900060E070E0CB010E943E060E947F070E9448
:100CA000440881E00C9417060895CF93FB01C2819C
:100CB000CC2309F19C0122513F452031310520F51B
:100CC00082510E945408C0E08C2FCF91089581E09A
:100CD0000E94301343E062E081E00E941403F3CFEE
:100CE00081E00E94511343E062E081E00E9414031E
:100CF000EBCF82E0F6CF8031FFE59F0789F38131AA
:100D00009F45B9F3C1E0E0CF8031EFE59E07F9F2EE
:100D100081319F45C9F682E0DBCF2FEFFC012083B4
:100D200008951F93CF93DF93EC01162FE881E150D4
:100D3000E33108F050C0F0E0EE50FC4D0C948D23F0
:100D4000198289E08A830FC08981823099F08330CB
:100D5000A1F08130B1F40E94E7160E9493236A83C8
:100D60007B838C839D83612FCE01DF91CF911F9177
:100D70000C949D1C0E943506F0CF80E00E949405E3
:100D8000E1CF612FCE010E948D06EDCF89818230A7
:100D9000C1F76A817B818C819D810E9493230E948F
:100DA0003E06E1CF4B816A8189810E9451079827D5
:100DB000892798279D838C83D6CF2C813D8132272C
:100DC000232732274B816A8189810E946A07CBCF12
:100DD0000E947F07C8CF8FEF8883C5CF0E94EF079F
:100DE0008983C1CF0E94F1079827892798279A8382
:100DF0008983B9CF6B8170E089819A81AE014C5FA4
:100E00005F4F9827892798270E94F407ACCF6B8102
:100E100070E089819A81AE014C5F5F4F98278927E6
:100E200098270E941A089FCF0E9444089CCF0E94D6
:100E30004507D6CF6B8170E089819A81AE014C5F06
:100E40005F4F9827892798270E9496078CCF6B8140
:100E500070E089819A81AE014C5F5F4F98278927A6
:100E600098270E94BB077FCF0E942F067CCF0E944D
:100E70009D1C2FEF81EE94E0215080409040E1F7DF
:100E800000C000000E9426176ECF84E00895640F12
:100E90007727771F860F972F911D880F991F8696AA
:100EA00008950F931F93CF93DF930E9447078C0100
:100EB0000E94AE23C82FD0E0DC2FCC27C8010196BA
:100EC0000E94AE239E01282BC901DF91CF911F9173
:100ED0000F9108950F931F93CF93DF93122F032F3A
:100EE0000E944707EC01602F0E94BC23612FCE01B6
:100EF0000196DF91CF911F910F910C94BC230F931A
:100F00001F93CF930CEA10E0C0E0F80125913491D3
:100F100040E060E08C2F0E946A070E5F1F4FCF5F9A
:100F2000C43099F7CF911F910F910895EF92FF92DE
:100F30000F931F93CF93DF93EC018A017C01E60EA0
:100F4000F71ECE018696CE15DF0539F4DF91CF91DD
:100F50001F910F91FF90EF900895C830D10540F494
:100F60000E94AE23F80180830F5F1F4F2196E9CFC7
:100F7000F8011082F9CFCF92DF92EF92FF920F9398
:100F80001F93CF93DF937C016A018C01060F171F1B
:100F9000EC01CE018696C017D10749F4DF91CF91BD
:100FA0001F910F91FF90EF90DF90CF900895C83080
:100FB000D10540F4FE01EE19FF09EC0DFD1D608125
:100FC0000E94BC232196E5CF843030F4762B21F4A7
:100FD00040E060E00C94510790E080E0089580E1EB
:100FE000089582ED93E00895EF92FF920F931F937F
:100FF000CF93DF93EC018A017C01E60EF71ECE0150
:101000008E96CE15DF0539F4DF91CF911F910F91A8
:10101000FF90EF900895C23D23E0D20740F40E9474
:10102000AE23F80180830F5F1F4F2196E8CFF801B0
:101030001082F9CFCF92DF92EF92FF920F931F931E
:10104000CF93DF937C016A018C01060F171FEC011F
:10105000CE018E96C017D10749F4DF91CF911F9131
:101060000F91FF90EF90DF90CF900895C23D23E065
:10107000D20740F4FE01EE19FF09EC0DFD1D608161
:101080000E94BC232196E4CFCF93DF93CEE2D0E041
:1010900060E0CE010E94BC232196C11584E0D807F0
:1010A000B9F7DF91CF910895DF92EF92FF920F93FE
:1010B0001F93CF93DF9300D000D0CDB7DEB7F82ECB
:1010C0008FE08F1540F08FEF93E00E94AE230EE289
:1010D00010E08823C1F00F900F900F900F90DF91D8
:1010E000CF911F910F91FF90EF90DF900895011520
:1010F00084E0180781F3C8010E94AE23811101C06A
:10110000FA940F5F1F4FF110F2CF19821A821B82DF
:101110001C82DD24D39478018FEFE81AF80AC80105
:101120000E94AE2389831A828823A9F29FEF980F29
:10113000933078F48A83D9820E5F1F4FC7010E94D3
:10114000AE238B83882339F2CE0101960E94BD0223
:10115000E2CF8701F9CF0F931F93CF93DF93C62F71
:10116000D42F022FFC0182818823C9F0609395015E
:101170000E94DB16909394018093930180E28C0F80
:10118000883008F050C0C77081E001C0880FCA9550
:10119000EAF7DF91CF911F910F910C94BA0C109147
:1011A0009501161335C080919301909194010E948E
:1011B000F316883C910560F5C0E2CD0F1D17B9F01C
:1011C00080E2810F883040F4177081E001C0880F01
:1011D0001A95EAF70E94C10CC83048F481E09D2FAF
:1011E000977001C0880F9A95EAF70E94BA0C802F79
:1011F0000E94A70CC830B8F4D77081E001C0880FF6
:10120000DA95EAF7DF91CF911F910F910C94C10C01
:1012100080E28C0F883038F4C77081E001C0880FFD
:10122000CA95EAF7EFCFDF91CF911F910F91089503
:101230009C01CB01233F4CE5340731F190F4283D6C
:10124000FCE53F07E9F0293D4CE5340769F1273D0E
:101250003C4579F426E241EE61EE0E94AB0880E065
:101260000895253FFCE53F07B9F090F0263F3C4547
:10127000B9F0FC0182818823D1F010929501089584
:1012800027E245EE65EEE9CF26E241EE60EEE5CFDE
:1012900027E245EE64EEE1CF26E241EE62EEDDCFDD
:1012A00027E245EE66EED9CF28E241E0EBCF81E0C0
:1012B0000895CF93DF93EC01FB018281882309F429
:1012C00019C1C230FCE5DF07C0F1C6319CE5D90782
:1012D00030F09E012A5F3C452930310570F50E94AF
:1012E00078159093160280931502C031ECE5DE0765
:1012F00009F4CFC008F05BC0C8308CE5D80709F40A
:10130000B6C088F5C430ECE5DE0709F4A8C0C0F427
:10131000C2308CE5D80709F49CC080911502826028
:10132000C330DC4509F498C08091150290911602F3
:101330000E9486150E94360F80E0DF91CF910895BC
:10134000809115028061C630ECE5DE0709F484C0A7
:10135000809115028860C730DC4508F47DC080911B
:101360001502806279C0CC308CE5D80709F489C0B9
:1013700070F4809115028C60CA30ECE5DE0709F448
:101380006BC008F478C0809115028E7F65C0CE30A6
:101390008CE5D80709F479C0809115028B7FCF3096
:1013A000DC4508F459C0809115028F7E55C0CB3FB3
:1013B000ECE5DE0709F457C030F5C3318CE5D807FA
:1013C00009F46FC078F4C131ECE5DE0709F465C0BB
:1013D000C231DC4509F0A8CF0E94360F809115027A
:1013E0008F773AC0C5318CE5D80709F462C008F49C
:1013F00076C0809116028160CA3FDC4509F094CF27
:101400008093160291CFCF3FFCE5DF0709F44DC072
:1014100088F4809116028D7FCD3F9CE5D90781F33A
:10142000809116028E7FCE3FDC4550F380911602EC
:101430008360E6CFC130FDE5DF0709F459C008F449
:1014400044C080E0C230DD4509F06ECF0E94041632
:101450006BCF8091150281608093150265CF8091DA
:1014600015028460F9CF809116028260C9CF809105
:1014700015028064F1CF0E94360F809115028068BA
:10148000EBCF809115028D7FE7CF80911502877F8A
:10149000E3CF809115028F7DDFCF809115028F7B86
:1014A000DBCF80911502837FD7CF809116028C7F8E
:1014B000A7CF8091150282FB992790F921E092270E
:1014C00090FB82F990FB83F9C7CF80911602982F89
:1014D000909591708E7F892B90FB81F991CF0E941E
:1014E000360F90911502892F97FB87F98058B4CF5A
:1014F00081E0ACCF81E021CFCF93DF93EB01863148
:101500009C4511F50E94B0149A81992399F08A7A2A
:1015100091E009F490E090939601811109C089E26D
:101520000E948B140E94FC1480E0DF91CF910895FB
:1015300085E3F6CF80919601811104C089E20E9473
:101540009214F0CF85E3FBCF81E0EFCF90939C0125
:1015500080939B010895E0919B01F0919C0130974D
:1015600021F00190F081E02D099480E00895E09150
:101570009B01F0919C01309721F00280F381E02DD6
:1015800009940895E0919B01F0919C01309739F006
:1015900022E0DC012C930480F581E02D099408956C
:1015A0002091990130919A012817390771F0909391
:1015B0009A0180939901E0919B01F0919C013097F1
:1015C00021F00680F781E02D09940895209197017C
:1015D000309198012817390771F090939801809302
:1015E0009701E0919B01F0919C01309721F00084DC
:1015F000F185E02D0994089585B7806885BF85B78A
:10160000806885BF0895089508950C94030B08958C
:101610000C94070B0E94FC0A0E94040B0C94050B0F
:1016200081E008950C94100B0E94D2160E949B0535
:101630000E9442060E944D170C94080B0F931F93B3
:10164000CF93DF93CDB7DEB72A970FB6F894DEBFFE
:101650000FBECDBF0E94A6050E94120B882309F47D
:101660003EC080E00E949405182F00919E0108174B
:10167000B1F18091F20181FD0E949A05012700FFDE
:101680002EC01E821F82117018870E94DB16816097
:10169000782F9A8789874E815F8168858A850E9425
:1016A0008B0B80919E0191E0892780939E010E947F
:1016B000DA180E94AB0A90919D01891709F10E94E6
:1016C000AB0A80939D012A960FB6F894DEBF0FBE39
:1016D000CDBFDF91CF911F910F910C9439038FEF04
:1016E00089838A831B820E94DB168160782F9D8309
:1016F0008C8349815A816B818D810E948B0BD7CF5E
:101700002A960FB6F894DEBF0FBECDBFDF91CF9102
:101710001F910F910895CF93DF93CDB7DEB72B972D
:101720000FB6F894DEBF0FBECDBF4F8358876987D1
:101730007A878B871E821D8285E0FE013796DE0147
:10174000119601900D928A95E1F749815A816B813A
:101750007C818D819E812B960FB6F894DEBF0FBEE3
:10176000CDBFDF91CF910C94AC11FC0180819181B0
:101770000C945D14CF93C82F882309F490C082384D
:10178000C1F40E94AB0A81FD8AC089E30E948B14D8
:101790000E94FC142FEF81EE94E021508040904095
:1017A000E1F700C0000089E30E949214CF910C94ED
:1017B000FC148338A1F40E94AB0A80FD70C083E55D
:1017C0000E948B140E94FC142FEF81EE94E02150B4
:1017D00080409040E1F700C0000083E5E5CF843809
:1017E000A1F40E94AB0A82FD5AC087E40E948B14C8
:1017F0000E94FC142FEF81EE94E021508040904035
:10180000E1F700C0000087E4CFCF8CEF8C0F813A66
:10181000B8F48C2F0E946B1B811141C06C2F8091FA
:101820000001909101010E941B16882329F08C2F42
:101830000E9492140E94FC148C2F0E948B14B6CF2D
:1018400080E28C0F883048F4C77081E001C0880FB7
:10185000CA95EAF70E94B314A9CFEBE5EC0FE33089
:1018600040F4F0E0EC58FE4F808190E0CF910C9472
:10187000D00AE8E5EC0FE73150F4F0E0EE0FFF1F7F
:10188000EA5BFE4F80819181CF910C94E60AC03FC4
:1018900030F08C2F0E94E817CF910C94CF18CF9185
:1018A0000895882309F452C0823871F40E94AB0A6B
:1018B00081FF4CC089E30E948B140E94FC1489E3D1
:1018C0000E9492140C94FC14833859F40E94AB0AC1
:1018D00080FF3CC083E50E948B140E94FC1483E5CA
:1018E000EFCF843859F40E94AB0A82FF2FC087E4FF
:1018F0000E948B140E94FC1487E4E2CF9CEF980FA7
:10190000913AF0F290E2980F983050F4877091E09D
:1019100001C0990F8A95EAF7892F0E94B914D2CF96
:101920009BE5980F933020F490E080E00C94D00A6F
:1019300098E5980F973120F490E080E00C94E60A47
:10194000803F20F00E9450180C94CF180895CF9338
:10195000C82F0E94BA0BC93349F42FEF87EE93E0EA
:10196000215080409040E1F700C000008C2FCF91C3
:101970000C94510C882321F00E94B3140C94FC1495
:101980000895882321F00E94B9140C94FC14089542
:10199000BF92CF92DF92EF92FF920F931F93CF935C
:1019A000DF936C01D62FC72FFC01058102950F70C4
:1019B000128111110E94D0140E94A914E82E8823CC
:1019C00091F01123D1F08C2F807F803421F080E2C0
:1019D0008D0F883090F082E00E9447150E94A91474
:1019E00091E0E82EE926BC2EB2949FE0B922EB2DBF
:1019F000F0E0EB5FFB4D0C948D23E12CF4CF0C2F2A
:101A00000F70C07F11F00295007F1123A9F0002311
:101A100059F080E28D0F883010F0D11109C0802F6D
:101A20000E94B3140E94FC148D2F0E94BA0B14C0A4
:101A3000802F0E94C314F6CF8D2F0E94510C0023DB
:101A400059F080E28D0F883010F0D1112CC0802F1A
:101A50000E94B9140E94FC142B2D2850330B243003
:101A6000310520F40E94AB0A0E943903EE2009F4EC
:101A70009EC10E94A51480FD9AC1F60112820E94A7
:101A80009F140E943013C6010E94F80E0E949F14FA
:101A9000DF91CF911F910F91FF90EF90DF90CF904A
:101AA000BF900C945113802F0E94C914D3CFFC2FE8
:101AB000FF70FF2EC07FC03219F0F29480EFF82241
:101AC000DD2369F0D13049F1112391F1002351F167
:101AD000F601858180FFA8CF8F70858323C01123F5
:101AE00081F0011106C00E94E3148F290E94BA0CF4
:101AF000B3CF0130C1F70E94E3148F290E94E9148B
:101B0000ABCF011106C00E94F2148F2D0E94C10CB0
:101B1000A3CF013009F4A0CFF6CF112329F006306E
:101B200008F09ACF8F2DE2CF053008F095CFEDCF9A
:101B3000002359F3D93349F4FFEF27EE33E0F15096
:101B400020403040E1F700C000008D2F0E94510C72
:101B500083CF8C2F86958695837069F0813009F04C
:101B60007BCF8D2F9C2F9370111102C090E080E0ED
:101B70000E94E60A71CF8D2F9C2F9370111102C025
:101B800090E080E00E94D00A67CF8D2F112329F0CA
:101B90000E94E8170E94CF185FCF0E945018FACF1A
:101BA0008C2F837009F041C0111156CF4D2F4295F3
:101BB00046954770440F440F0D2F0F7010E030E032
:101BC00020E0042E04C0000F111F221F331F0A94AF
:101BD000D2F760E070E0CB01D4FF0FC06FE070E09F
:101BE00080E090E004C0660F771F881F991F4A9518
:101BF000D2F76095709580959095C695C695C370FF
:101C0000602B712B822B932BC23049F058F4C130DA
:101C100019F00E94E21220CF0E94D0121DCF0E9424
:101C2000F4121ACF0E94CE1217CF8695112311F00D
:101C30008C2F8170882309F40FCF4D2F4295469544
:101C40004770440F440F0D2F0F7010E030E020E07C
:101C5000042E04C0000F111F221F331F0A94D2F755
:101C600060E070E0CB01D4FF0FC06FE070E080E077
:101C700090E004C0660F771F881F991F4A95D2F71E
:101C80006095709580959095C695C695C370602BAC
:101C9000712B822B932BC23049F058F4C13019F0CC
:101CA0000E94A713D9CE0E949513D6CE0E94B913D5
:101CB000D3CE0E940A13D0CECF70112329F08C2FDF
:101CC0000E9430138D2F12CF8D2F0E94C10C8C2FAC
:101CD0000E945113C1CED23F89F160F4D03FC9F0C8
:101CE000D13F29F1112309F442C001119DCE8C2F5F
:101CF0008F7121C0D33F39F1D43FA1F7112369F18E
:101D0000CF718C2F0E94301363E08C2F0E9432150C
:101D1000A3CE112341F0053008F09ECE8C2F8F7199
:101D20000E94741399CE063008F096CEF7CF8C2F10
:101D30008F71112369F20E9430138ECE8C2F8F7118
:101D40001123C9F3C5CF112329F08C2F8F710E9465
:101D50001B1382CE0E9416137FCE81E00E9447158E
:101D6000023008F479CE82E00E94471575CE002338
:101D700059F0D93309F0E9CE8FEF97EEE3E08150C7
:101D80009040E040E1F7DFCE8C2F8F71A1CF4C2F38
:101D90004F706D2FC6010E9493030E9446125CCEC5
:101DA0004C2F4F706D2FC6010E94960355CEDF91C8
:101DB000CF911F910F91FF90EF90DF90CF90BF9048
:101DC00008950F931F93CF93DF93EC01688179817E
:101DD0008A810E9467148C010E94CB130E94CD124D
:101DE000B801CE01DF91CF911F910F910C94C80CD7
:101DF000CF93DF93EC018B819C81892B29F0888123
:101E0000998189238F3F59F4DF91CF910895CE01B5
:101E10000E94E10ECE01DF91CF910C94FE01CE0124
:101E20000E9451038111F3CF0E94A914882361F30A
:101E30008A81882349F382E0DF91CF910C94471582
:101E40000E94D0140E94E0140E94FC140E94F41915
:101E50000E94CF1890E080E00E94D00A90E080E0DD
:101E60000C94E60A0E9499140C94200F0E94C0144E
:101E70000C94320FE92FE295EF70E250EE3070F4DF
:101E8000F0E0EB5EFB4D0C948D23803F19F020F4C5
:101E9000883E20F481E00895843FE1F380E00895D6
:101EA000883EC0F3813FD1F7F5CF93FB882780F9B7
:101EB00008950E945D140C943A0FCF93DF9300D0E5
:101EC00000D00F92CDB7DEB70F900F900F900F900C
:101ED0000F90DF91CF910895CF93DF9300D000D082
:101EE00000D0CDB7DEB726960FB6F894DEBF0FBE92
:101EF000CDBFDF91CF9108951F93CF93DF93C09112
:101F0000A00116E08091A1018C1304C0DF91CF9154
:101F10001F910895D0E01C9FF0011D9FF00D11242A
:101F2000EE55FE4F4081518162817381848195819C
:101F30000E946C0F2196C770E5CF4091D20150915D
:101F4000D3016091D4017091D5018091D601909117
:101F5000D7010C946C0F1F93CF93DF938091D7011F
:101F6000807FA9F48091D401882389F08091A00119
:101F7000C091A1016091D2017091D301A091D501CE
:101F8000B091D601D62FD72316E0C81304C0DF9135
:101F9000CF911F91089590E0109711F0DF3F19F451
:101FA00001968770F2CF189F9001199F300D112470
:101FB000F901EE55FE4F41814713F2CF40814613A0
:101FC000EFCF42814111ECCF438154814A1B5B0B1F
:101FD000483C510528F78091D7018F70806180932C
:101FE000D701F901E955FE4F80818F7080618083B0
:101FF00082ED91E00E94F80EDF91CF911F910C9439
:102000007C0FAF92BF92CF92DF92EF92FF920F932D
:102010001F93CF93DF93CDB7DEB761970FB6F894D8
:10202000DEBF0FBECDBF8C0185E0F801DE011D963D
:1020300001900D928A95E1F7F80140815181E2808B
:1020400082EDC82E81E0D82E6091D5017091D60125
:102050006115710509F461C19091D2012091D301FC
:10206000892F82238F3F09F458C1A380B480F09058
:10207000D401F501E61BF70BFF2009F4FCC08091A9
:10208000D701382F307FE83CF10508F0B2C031119C
:1020900079C0FE2C251323C0941321C0E1101FC06A
:1020A0008F7080618093D7010E949D0FC6010E94AE
:1020B000F80E8091D701F80185838F2D61960FB6B8
:1020C000F894DEBF0FBECDBFDF91CF911F910F916E
:1020D000FF90EF90DF90CF90BF90AF900895AB2826
:1020E00029F0842F85238F3F09F033C180E0F82F3A
:1020F000F170DF2E80FF3CC08091A0012091A101F2
:1021000036E0821315C04D875E878D859E850E94BF
:102110005D14292F22952F702230F0F0243018F50D
:102120009F70F1F0F8019581907FD1F4D12C1EC001
:1021300090E0389FF001399FF00D1124EE55FE4FCD
:102140006181651306C06081641303C062816E11F2
:102150000FC001968770D5CF9F7011F0882331F39F
:10216000805E883018F3C8010E94F80EFD2CA5CFC0
:10217000EE2009F4A2CF8091D70181608093D7012E
:10218000F12C9BCF251306C0941304C0F801EE2058
:1021900009F48DC04D875E878D859E850E94590FFD
:1021A000882319F1EE2009F18091D701803270F077
:1021B0002091D2013091D30138872F831986BB86B5
:1021C000AA868C87CE0107960E94F80E86E0F80159
:1021D000A2EDB1E001900D928A95E1F70E94AB0F5C
:1021E0000E949D0FFF24F39468CFC8010E94F80E4F
:1021F000F9CF311113C07A2DB98AA88A6E2D898939
:102200000E945D0F82ED91E00E94F80E86E0F601DB
:1022100011928A95E9F70E949D0FB2CF25130FC046
:1022200094130DC0E1100BC0F8018583C8010E9412
:10223000F80E86E0F60111928A95E9F73ECF4D87B8
:102240005E878D859E850E94590F882371F2EE204E
:1022500061F28091D701803208F4B8CF2091D20189
:102260003091D3013A8329831B82BD82AC828E8355
:10227000CE010196A9CFE83CF10508F041C0FE2C43
:10228000EE2009F4B2CF25132AC0941328C0809100
:10229000D70180FD1BC0982F907FC1F0F801858386
:1022A000903F31F0982F907F905F8F70892B8583BE
:1022B000C8010E94F80E86E0F801A2EDB1E001909D
:1022C0000D928A95E1F70E949D0FF7CE86E0F80106
:1022D000A2EDB1E001900D928A95E1F7EECE4D8727
:1022E0005E878D859E850E94590F81116FCF8091E9
:1022F000D70181608093D701C8010E94F80EDDCE1E
:102300007A2DB98AA88A6E2D89890E945D0F86E090
:10231000F60111928A95E9F7D6CFEE2009F465CF40
:102320004D875E878D859E850E94590FF82E8823E4
:1023300009F45BCF86E0F801A2EDB1E001900D92C7
:102340008A95E1F782ED91E00E94B50B0E94AB0FF8
:10235000BACF81E08E25CBCE1F93CF93DF93CDB73D
:10236000DEB72C970FB6F894DEBF0FBECDBF4F83FC
:10237000588769877A878B879C87CE0107960E944A
:102380000110882369F08A859B85892B39F04F815C
:102390005885842F85238F3F09F071C016E05FC0F8
:1023A00086E0FE013796DE01119601900D928A9526
:1023B000E1F78A859B85892B89F38F81988589230D
:1023C0008F3F61F32091A10130E0C9010196877030
:1023D00099274091A0014817190671F40E94360F01
:1023E0001092A1011092A00186E0E2EDF1E0DF0180
:1023F0001D928A95E9F7D2CF96E0929FD001939FE4
:10240000B00D1124AE55BE4FFE01319601900D92D4
:102410009A95E1F78093A1010E947C0FBFCF819F25
:10242000C00111248E559E4F0E9401108823E9F0AF
:10243000E091A0011E9FF0011124EE55FE4F408156
:10244000518162817381848195810E946C0F80919A
:10245000A00190E00196877099278093A001809158
:10246000A0019091A1018913DACF2C960FB6F894B0
:10247000DEBF0FBECDBFDF91CF911F91089569855B
:102480007A858B859C850E946C0F88CFEF92FF9296
:102490000F931F93CF93DF938C01892B81F0F12C45
:1024A000EE24E394E8012196F8018491843770F4D6
:1024B000843008F05FC08130B1F08230A1F1DF914B
:1024C000CF911F910F91FF90EF900895853709F4F8
:1024D0004CC008F43DC09CE7980F903780F78F7789
:1024E0000E94510C49C00E5F1F4FFE01849190E283
:1024F000980F983060F48770FE2D01C0FF0F8A9509
:10250000EAF78F2F0E94D3140E94FC1402C00E948D
:10251000BA0B8F2D815030F2EFE9FFE03197F1F7E0
:1025200000C00000F7CF0E5F1F4FFE01849190E2C4
:10253000980F983050F48770FE2D01C0FF0F8A95D8
:10254000EAF78F2F0E94D914DFCF0E94510CE1CF00
:102550000E5F1F4FFE01C491C150D8F28FE99FE07A
:102560000197F1F700C00000F7CF0E5F1F4FFE018B
:10257000F490CFCF0E94BA0B8E01CBCF08950C946C
:10258000BE120E94BF126093E1017093E20180933A
:10259000E3019093E4010C94200F08950C94C11270
:1025A0000F931F930091E1011091E2012091E3014B
:1025B0003091E401602B712B822B932B1F910F9193
:1025C0000C94C1120F931F930091E1011091E2014D
:1025D0002091E3013091E40160237123822393234E
:1025E0001F910F910C94C1120F931F930091E10161
:1025F0001091E2012091E3013091E40160277127FD
:10260000822793271F910F910C94C1120C94BE1234
:102610000C9406130E9408136093DD017093DE0191
:102620008093DF019093E0010C94200F60E070E054
:10263000CB010C940A130F931F9341E050E060E02C
:1026400070E08A019B0104C0000F111F221F331F7D
:102650008A95D2F7C901B8011F910F910C940A1302
:102660000F931F9341E050E060E070E004C0440F1E
:10267000551F661F771F8A95D2F78091DD019091D3
:10268000DE01A091DF01B091E0018A019B01082BDE
:10269000192B2A2B3B2BC901B8011F910F910C94C8
:1026A0000A130F931F9341E050E060E070E004C014
:1026B000440F551F661F771F8A95D2F7CB01BA01C9
:1026C00060957095809590950091DD011091DE01E7
:1026D0002091DF013091E001602371238223932355
:1026E0001F910F910C940A130F931F9341E050E038
:1026F00060E070E004C0440F551F661F771F8A9585
:10270000D2F78091DD019091DE01A091DF01B091BF
:10271000E0018A019B01082719272A273B27C901C5
:10272000B8011F910F910C940A130F931F930091FE
:10273000DD011091DE012091DF013091E001602B7D
:10274000712B822B932B1F910F910C940A130F93D3
:102750001F930091DD011091DE012091DF01309186
:10276000E00160237123822393231F910F910C9426
:102770000A130F931F930091DD011091DE01209148
:10278000DF013091E00160277127822793271F9195
:102790000F910C940A130895980F892F877041E0C8
:1027A00001C0440F8A95EAF796959695969585E02F
:1027B000989FF0011124E852FE4F30E020E070E0D5
:1027C0005191DF011197CB01022E02C0969587959A
:1027D0000A94E2F7817081958527842385278C935D
:1027E0002F5F3F4F2530310559F70895980F692F16
:1027F000677096959695969585E0989FF0011124BF
:10280000E852FE4F50E040E080E0219130E0062E9B
:1028100002C0369527950A94E2F721703327042EDB
:1028200001C0220F0A94EAF7822B4F5F5F4F4530B9
:10283000510559F70895BF92CF92DF92EF92FF9220
:102840000F931F93CF93DF938C01C090DD01D09045
:10285000DE01E090DF01F090E0018091E1019091D4
:10286000E201A091E301B091E401C82AD92AEA2A41
:10287000FB2ACFE1D0E0BC2ED701C6010C2E04C04C
:10288000B695A795979587950A94D2F780FD0EC0C7
:10289000219788F7B12C8B2DDF91CF911F910F914C
:1028A000FF90EF90DF90CF90BF900895B8018C2FEC
:1028B0000E949F03019761F3EECFCF93DF93EC016A
:1028C0000E941B14BE01DF91CF910C949F031F93B4
:1028D000CF93DF93EB0190919F01992331F0CB01CE
:1028E000DF91CF911F910C945D14882379F0CB0177
:1028F0000E941B14182F682FCE010E94CC13BE011A
:10290000812FDF91CF911F910C949F03CB010E94E7
:10291000F613182FF4CF682F8091000190910101D8
:102920000C945116682F80910001909101010C9434
:10293000531680910001909101010C9455168091DD
:10294000E50185958595859508958091E5018770C8
:1029500008959091E501977081E009F480E0089571
:102960008091F10108959091F101892B8093F101FB
:10297000089580959091F10198239093F101089525
:102980001092F10108959091F001892B8093F0014C
:10299000089580959091F00198239093F001089507
:1029A0001092F00108959091EF01892B8093EF012F
:1029B000089580959091EF0198239093EF010895E9
:1029C0001092EF0108958091E601089508950C9406
:1029D000E6149091E601981721F08093E6010C949B
:1029E000E71408958091E601882329F01092E6010A
:1029F00080E00C94E7140895E0910001F09101014A
:102A00008091F1018083E0910001F09101018081CA
:102A10009091F001892B8083E0910001F0910101F8
:102A200080819091EF01892B80839091E601992319
:102A300081F0E0910001F09101018081892B808378
:102A400080910001909101010E94091681110E945C
:102A5000F21480910001909101010C94B70A08953D
:102A60000C942F1598E0899F90011124622B60939C
:102A7000E5010E9430138091E50185958595859546
:102A80000C9430151092E50180E00C943015909173
:102A9000E501809589238093E501282F277071F443
:102AA000282F082E000C330B9217130639F085954A
:102AB000859585950E9451130C94421508956FEFEA
:102AC0007FEF90E080E00C94DA2390E080E00E94B9
:102AD000B62321E08C3E9E4F09F020E0822F08951E
:102AE00082E090E00C94AE2383E090E00C94AE235F
:102AF000CF9384E090E00E94AE23C82F81E290E063
:102B00000E94AE23982F8C2FCF910895CF93C92F79
:102B1000682F84E090E00E94BC236C2F81E290E05B
:102B2000CF910C94BC23AB01BC018FE090E00C94DE
:102B3000CE23AB01BC0183E190E00C94CE2360E096
:102B400070E0CB010C94991560E070E0CB010E941D
:102B500093150C949F156CEE7EEF90E080E00E9440
:102B6000DA2360E082E090E00E94BC2360E083E032
:102B700090E00E94BC231092E1011092E2011092B9
:102B8000E3011092E40160E084E090E00E94BC2345
:102B900060E081E290E00E94BC2360E085E090E08C
:102BA0000E94BC2360E086E090E00E94BC236FEFAF
:102BB00087E090E00E94BC2340E050E0BA0188E04A
:102BC00090E00E94CE2360E08DE090E00E94BC2364
:102BD00040E050E0BA0188E190E00E94CE2360E03E
:102BE00087E190E00E94BC2340E050E0BA018CE114
:102BF00090E00E94CE2360E080E290E00E94BC233F
:102C00000C94A4150C94AB15682F8EE090E00C94F6
:102C1000BC239C012E5F3F4FAC01485F5F4F80E0BB
:102C20002417350709F40895F90191919F0199231B
:102C3000B9F38F5FF5CF662349F0FC013296089611
:102C40002191261729F0E817F907D1F780E00895B8
:102C500081E008959C01FC0132969FEF80E0419154
:102C6000461751F09F3F19F4411101C0982F8F5F13
:102C70008630A9F79F3F09F40895290F311D97FD6C
:102C80003A95F90162830895FC01329608962191E4
:102C9000261303C0DF0111971C92E817F907B9F753
:102CA00008950C942A160C944416029626E0FC0112
:102CB00011922A95E9F70895089508950C945D16E8
:102CC0000E945E1680911B02843049F11092F3013C
:102CD00088E190E020E40FB6F894A8958093600016
:102CE0000FBE2093600080E00E9439030E945E16B0
:102CF00083B7817F846083BF83B7816083BF78940B
:102D0000889583B78E7F83BF0FB6F894A89580917E
:102D10006000886180936000109260000FBE08958B
:102D200008950E945C160E94A6050E94901680E0FD
:102D30000E94940591E0811101C090E0892F0895CF
:102D400008950C94A0160E94360F0E94AB0A0E94B0
:102D500039030C94A1161F921FB61F9211248F9352
:102D60009F93AF93BF938091F301811113C0809122
:102D7000110290911202A0911302B0911402419697
:102D8000A11DB11D8093110290931202A093130212
:102D9000B0931402BF91AF919F918F911F901FBE6E
:102DA0001F90189582E084BD93E095BD9AEF97BD82
:102DB00080936E0008952FB7F8948091110290913E
:102DC0001202A0911302B09114022FBF08952FB7E1
:102DD000F894609111027091120280911302909107
:102DE00014022FBF08959C014FB7F89480911102EF
:102DF00090911202A0911302B09114024FBF821B56
:102E0000930B089578941F921FB61F9211248F93ED
:102E10009F93AF93BF938091110290911202A09162
:102E20001302B09114020196A11DB11D80931102ED
:102E300090931202A0931302B0931402BF91AF912A
:102E40009F918F911F901FBE1F90189587E797E75E
:102E5000909301088093000888E19AE00FB6F894F7
:102E6000A895809360000FBE90936000FFCF0C94F4
:102E70002F060E94A6058FE39CE90197F1F700C099
:102E800000000E94A60580E00E94940580FF04C017
:102E90000E9437170C94261708950E94651581111A
:102EA00002C00E9402160E9470158093F2010E94D7
:102EB000781590931602809315020E947415682F5E
:102EC00070E090E080E00C94CE128091FB0180FFD6
:102ED00012C06091070185E0689FB00111247595CB
:102EE00067957595679560387105A8F56115710549
:102EF000A1F1862F089581FF09C06091070185E047
:102F0000689FB001112475956795EDCF6091070119
:102F100082FD0AC08091FA018823D1F090910601C8
:102F200060910701891728F085E0689FB00111249E
:102F3000DACF869FB001112485E0869F9001879F9C
:102F4000300D1124692F70E0C9010E947923CBCF85
:102F500065E070E0CECF8FE7089581E0089580911D
:102F6000FB0180FF0CC06091030170E075956795CF
:102F7000759567956115710549F1862F089581FF53
:102F800006C06091030170E075956795F3CF60917D
:102F9000030182FD0BC09091FA019923A1F0609189
:102FA000020180910301961738F0682F70E06038B5
:102FB000710500F38FE70895899FC001112470E027
:102FC0000E947923F4CF61E070E0D7CF81E00895CB
:102FD000803F31F40E94651781958093FF01089529
:102FE000813F19F40E946517F8CF823F31F40E94A7
:102FF000651781958093FE010895833F19F40E941F
:103000006517F8CF893F29F40E94AF17809300021B
:1030100008958A3F21F40E94AF178195F7CF8B3F27
:1030200031F40E94AF1781958093010208958C3F7F
:1030300019F40E94AF17F8CF843F31F48091FD015D
:1030400081608093FD010895853F21F48091FD0109
:103050008260F7CF863F21F48091FD018460F1CF3B
:10306000873F21F48091FD018860EBCF883F21F4F8
:103070008091FD018061E5CF8D3F31F48091FB01AE
:1030800081608093FB0108958E3F21F48091FB01C4
:103090008260F7CF8F3FB9F78091FB018460F1CF59
:1030A0009091FE01803F41F48091FF0187FD1092D5
:1030B000FF01992371F00895813F29F48091FF0168
:1030C0001816ACF3F6CF823F81F497FFF2CF10923F
:1030D000FE018091FF0190910002892B90910102E5
:1030E000892B49F71092FA010895833F19F41916B4
:1030F00074F3DFCF893F39F4809100021816CCF6C3
:1031000010920002D6CF8A3F29F48091000287FFF7
:10311000D0CFF6CF8B3F39F48091010287FFC9CF22
:1031200010920102C6CF8C3F29F48091010218163B
:10313000BCF3BFCF843F31F48091FD018E7F80933B
:10314000FD01B7CF853F21F48091FD018D7FF7CF41
:10315000863F21F48091FD018B7FF1CF873F21F4E1
:103160008091FD01877FEBCF883F21F48091FD01A5
:103170008F7EE5CF8D3F31F48091FB018E7F809370
:10318000FB0197CF8E3F21F48091FB018D7FF7CF1C
:103190008F3F09F08ECF8091FB018B7FF0CF8CEFBA
:1031A00091E00E94C20A0E94DB169093F90180937D
:1031B000F8010895CF93DF9300D000D000D0CDB7B1
:1031C000DEB786E0ECEFF1E0DE01119601900D92A2
:1031D0008A95E1F78091FE019091FF01892B81F0A2
:1031E0008091F6019091F7010E94F316AC01909145
:1031F000FA01992331F1809108018417150670F1C5
:103200008091000290910102892B91F08091F4014C
:103210009091F5010E94F316AC019091FA01992367
:1032200009F478C0809104018417150608F480C061
:1032300026960FB6F894DEBF0FBECDBFDF91CF91BB
:103240000895209109018AE0289F900111242417F4
:103250003507B0F69F5F9093FA0102C09F3FD1F708
:1032600010920002109201028091FE01181624F4BF
:103270000E9465178093FE018091FE0187FF05C0C3
:103280000E94651781958093FE018091FF011816B9
:1032900024F40E9465178093FF018091FF0187FF4E
:1032A00005C00E94651781958093FF013091FE0152
:1032B0003323A1F02091FF01222381F045EB340359
:1032C000C00111249923F1F09093FE0145EB2403F2
:1032D000900111243323D1F03093FF010E94CF18C5
:1032E0008091F8019091F9019093F7018093F60194
:1032F00086E0FE013196ACEFB1E001900D928A9527
:10330000E1F77ECF81E08093FE01E0CF81E0809302
:10331000FF01E4CF209105018AE0289F900111244C
:103320002417350708F084CF9F5F9093FA0102C0FD
:103330009F3FD1F71092FE011092FF018091000291
:10334000181624F40E94AF178093000280910002A7
:1033500087FF05C00E94AF1781958093000280917E
:103360000102181624F40E94AF1780930102809185
:10337000010287FF05C00E94AF178195809301026B
:10338000309100023323A1F020910102222381F029
:1033900045EB3403C00111249923F1F0909300020E
:1033A00045EB2403900111243323D1F03093010223
:1033B0000E94CF188091F8019091F9019093F50146
:1033C0008093F40186E0FE013196ACEFB1E001900C
:1033D0000D928A95E1F72CCF81E080930002E0CF37
:1033E00081E080930102E4CF86E0ECEFF1E0DF01C1
:1033F0001D928A95E9F71092FA011092FB01089547
:10340000833081F128F4813059F08230D1F0089571
:10341000853009F449C0B8F1863009F456C00895E2
:1034200080910901482F460F5527551F4F3F5105E1
:1034300024F4680F6093090108958FEF80930901C8
:10344000089580910801482F460F5527551F4F3F7B
:10345000510524F4680F6093080108958FEF80935D
:103460000801089580910701482F460F5527551FE1
:103470004F3F510524F4680F6093070108958FEFC3
:1034800080930701089580910601482F460F552724
:10349000551F4F3F510524F4680F609306010895AE
:1034A0008FEF80930601089580910301482F460F06
:1034B0005527551F4F3F510524F4680F60930301B2
:1034C00008958FEF80930301089580910201482FA2
:1034D000460F5527551F4F3F510524F4680F609341
:1034E000020108958FEF809302010895833011F156
:1034F00028F4813049F0823091F00895853081F1CF
:1035000020F18630C1F1089580910901681720F4F7
:10351000861B8093090108951092090108958091F6
:103520000801681720F4861B809308010895109203
:103530000801089580910701681720F4861B809385
:1035400007010895109207010895809106016817F8
:1035500020F4861B809306010895109206010895B9
:1035600080910301681720F4861B8093030108955E
:1035700010920301089580910201681720F4861BC0
:103580008093020108951092020108950F931F93F2
:1035900041E050E060E070E08A019B0104C0000F50
:1035A000111F221F331F8A95D2F7C901B8010E944B
:1035B000CE121F910F910C94360F8B3109F461C01C
:1035C00040F58B3071F078F4863009F443C020F474
:1035D000853059F180E00895873009F444C088307F
:1035E000C9F781E00895803109F459C068F48E303C
:1035F00089F79091F201892F8B7F92FF84608093ED
:10360000F20182FD48C0EDCF863159F3893149F38B
:10361000E1CF8A32E1F060F48732A9F020F48E31F4
:10362000C8F28D5111C08932A9F60E944203D9CF48
:10363000833438F48A33F0F5853329F0883389F2FE
:10364000C9CF833439F680E00E94C61ACACF0E94DF
:103650000216C7CF8091F201807F8093F20181E052
:103660008093030208959091F201892F8E7F90FF3D
:1036700081608093F20180FDB4CF817F8093F2015D
:10368000B0CF9091F201892F8D7F91FF826080935E
:10369000F20181FFA6CF8091F2018160EFCF90917E
:1036A000F201892F877F93FF88608093F20183FD69
:1036B000F2CF97CF8953C8CF80E008950C945C1B5C
:1036C0008E518A3030F4E82FF0E0E958FE4F8081C7
:1036D000089580E00895CF93C82F80910302813030
:1036E000B9F0882331F08230A1F11092030280E01A
:1036F0000DC00E94B0148232D1F78C2F0E945C1B47
:1037000081111BC08C2F0E94DD1A8170CF9108950A
:103710000E94B014823289F38C2F0E945E1B8111AB
:103720000AC0C43199F060F4CB3029F0C03169F798
:1037300082E08093030281E0E8CF81E090E0E5CF72
:10374000C93221F0C833B9F380E0DFCF1092030211
:10375000FBCFC93219F188F4C43101F120F4C7302C
:1037600081F181E0D3CF82EE8C0F8630D0F78C2FA1
:103770000E94601B80930202F4CFCE3401F140F42A
:103780006AE0CB3471F7809102020E94001AE9CFFF
:10379000C13579F061E0C235B1F3E3CF8091020227
:1037A000882319F010920202DCCF81E0809303029B
:1037B000ADCF61E0809102020E94761AD2CF6AE01A
:1037C000F9CF8EE18093090182E3809308018AE0BA
:1037D0008093070184E18093060188E080930301D0
:1037E00088E280930201BDCF80910C020895CF93AF
:1037F000DF9300D00F92CDB7DEB790911B029430CB
:1038000011F589837B836A839093E9008FEF909110
:10381000E800815095FD06C095ED9A95F1F70000FE
:103820008111F5CF8091E80085FF0DC050E040E0A8
:1038300063E070E0CE0101960E94991E8091E8003D
:103840008E778093E8000F900F900F90DF91CF91CB
:103850000895CF93DF93EC010E947C1E823011F01B
:10386000843031F4BE0184E0DF91CF910C94F71BDA
:10387000DF91CF910895BC0183E00C94F71BCF93A7
:10388000DF93EC010E947C1E823011F08430F9F449
:1038900084E08093E9008FEF9091E800815095FDDE
:1038A00006C095ED9A95F1F700008111F5CF809152
:1038B000E80085FF0CC050E040E066E070E0CE011B
:1038C0000E94991E8091E8008E778093E800DF9136
:1038D000CF910895CF93DF93EC010E947C1E82303C
:1038E00011F0843039F581E08093E9008FEF9091F9
:1038F000E800815095FD06C095ED9A95F1F700001E
:103900008111F5CF8091E80085FF14C050E040E0C0
:1039100068E070E0CE010E94991E8091E8008E77E9
:103920008093E80088E0FE01A4E0B2E001900D92EF
:103930008A95E1F7DF91CF910895CF93FC01603232
:1039400021F580911B02843001F5C091E900CF7010
:103950002091EC00922F917020FD90E8C92B82E01D
:103960008093E9008091E80080FF0CC050E040E0C7
:1039700060E270E0CF010E94991E8091E8008E778E
:103980008093E800CF70C093E900CF9108958091B3
:103990001A02811109C00E9478200E94D5208091CE
:1039A000E20084608093E200089510921A02089564
:1039B000089508950C94A31642E061EC81E00E9402
:1039C000F41F42E261EC84E00E94F41F42E261ECE9
:1039D00082E00E94F41F42E260EC83E00C94F41F4A
:1039E00080911D02833009F461C030F48130D1F13F
:1039F000823009F49DC008958A3009F489C08B3063
:103A000009F46FC0893009F050C080911C028132E6
:103A100009F04BC08091200290912102009719F08B
:103A2000029709F042C08091E800877F8093E80008
:103A30008091E80082FF35C09091F3008091F20000
:103A4000029729F48091F1008B7F813021F48091DD
:103A5000F10080930C028091E8008B778093E8005E
:103A60000C94282080911C02813AF9F48091E8009E
:103A7000877F8093E8008091200290912102892B1A
:103A800061F468E084E092E070E00E94371F80916A
:103A9000E8008B778093E800089560E090E080E094
:103AA000F3CF80911B028111C3CF089580911C0236
:103AB000813AD9F78091200290912102892BA9F7B0
:103AC0008091E800877F8093E8008091E80080FF84
:103AD000FCCF809114018093F1008091E8008E77F3
:103AE000BDCF80911C02813201F78091200290911C
:103AF0002102892BD1F68091E800877F8093E8002E
:103B00000E94282080911E02809314010C94360F8D
:103B100080911C02813249F68091E800877F809372
:103B2000E8000E94282080911F0280930D020895D2
:103B300080911C02813A09F0B8CF8091E800877F1C
:103B40008093E8008091E80080FFFCCF80910D0217
:103B5000C2CFCDB7DEB7A0970FB6F894DEBF0FBEC9
:103B6000CDBF84B7877F84BF0FB6F894A8958091A6
:103B70006000886180936000109260000FBE80E852
:103B800090E00FB6F89480936100909361000FBEAF
:103B90000E940A0B0E9478200E94D5208091E200AA
:103BA00084608093E20078940E945E230E94140B4C
:103BB0008AE091E00E94A60A13E080911B02853002
:103BC00039F10E941E0B80911B028430B1F71093D3
:103BD000E9008091E80082FFF0CF8091E80090E05A
:103BE00085FF09C050E040E060E270E0CE01019640
:103BF0000E94E81E91E08091E8008B778093E800B6
:103C00009923D9F260E2CE0101960E949106D5CFA8
:103C10000E94601680911902882379F20E94911601
:103C2000882359F20E94831EC8CF0C94171E292F97
:103C300033272330310521F168F42130310509F4AF
:103C400049C02230310509F44AC090E080E030E0FC
:103C500020E029C02132310581F122323105A9F756
:103C60006330710590F7FB01EE0FFF1FEC57FE4F1D
:103C7000208131816F577E4FFB01808190E013C01E
:103C800099278130910599F0009741F08230910594
:103C900089F00397D1F6E4E5F1E002C0ECE8F1E049
:103CA000849190E09F01FA01318320830895EAE630
:103CB000F1E0F6CFEAE5F1E0F3CF6330710528F6E5
:103CC000660F771FFB01E657FE4F2081318189E0A7
:103CD00090E0E9CF82E190E02BEE31E0E4CF8BE59C
:103CE00090E020E931E0DFCF80911B02843011F4B5
:103CF00082E0089581E0089580910E02811102C052
:103D00000C94741E089580E189BD82E189BD09B4D7
:103D100000FEFDCF8091D8008F7D8093D8008091E8
:103D2000E00082608093E0008091E00081FDFCCFA4
:103D30000895AF92BF92CF92DF92FF920F931F939D
:103D4000CF93DF936C01EB018A010E944720F82E8C
:103D5000811123C00115110539F0F801808191818D
:103D6000C81BD90BC80ED91EB12CA12C2097A9F0C5
:103D70008091E80085FD22C08091E8008E778093D5
:103D8000E80001151105A1F0F80180819181A80ECC
:103D9000B91EB182A08285E0F82E8F2DDF91CF91E0
:103DA0001F910F91FF90DF90CF90BF90AF9008953B
:103DB0000E9447208823D1F2F82EEFCFF60181919F
:103DC0006F018093F1002197FFEFAF1ABF0ACECFAA
:103DD000AF92BF92CF92DF92FF920F931F93CF9338
:103DE000DF936C01EB018A010E944720F82E8111BC
:103DF00023C00115110539F0F80180819181C81B9C
:103E0000D90BC80ED91EB12CA12C2097A9F08091F6
:103E1000E80085FD22C08091E8008B778093E80060
:103E200001151105A1F0F80180819181A80EB91E3C
:103E3000B182A08285E0F82E8F2DDF91CF911F9166
:103E40000F91FF90DF90CF90BF90AF9008950E94A8
:103E500047208823D1F2F82EEFCF8091F100F601B0
:103E600081936F012197FFEFAF1ABF0ACECFFC01FC
:103E7000809122029091230286179707A0F0611586
